:020000040000FA
:100000000C9463000C948B000C948B000C948B006C
:100010000C948B000C94FC170C948B000C948B00AC
:100020000C948B000C948B000C948B000C948B0024
:100030000C948B000C948B000C948B000C948B0014
:100040000C9493160C948B000C9461160C943B1634
:100050000C948B000C948B000C948B000C948B00F4
:100060000C94DD160C948B00000000002400270087
:100070002A0000000000250028002B0000000000DE
:1000800023002600290004040404040404040202DA
:100090000202020203030303030301020408102007
:1000A0004080010204081020010204081020000012
:1000B0000008000201000003040700000000000027
:1000C000000049186F2A11241FBECFEFD8E0DEBF11
:1000D000CDBF25E0A0EAB3E001C01D92A83CB20765
:1000E000E1F713E0A0E0B1E0E6E2F2E602C005903D
:1000F0000D92A03AB107D9F710E0C2E6D0E004C0F3
:100100002197FE010E948B2DC136D107C9F70E94AD
:1001100055190C9406310C9400008091F5039091D0
:10012000F603891B990B08952F923F924F925F928D
:100130006F927F928F929F92AF92BF92CF92DF92F7
:10014000EF92FF920F931F93CF93DF93CDB7DEB75C
:1001500065970FB6F894DEBF0FBECDBF2D833E83EB
:100160004F83588769877A878B879C87A982BF8648
:10017000C88AD98AEA8AFB8A0C8B1D8B9E868D865B
:10018000211506ED300701E140070EE7500703E0B7
:10019000600771058105910511F008F009C12F373D
:1001A000304F4A4F5240610571058105910509F0B4
:1001B00008F469C19501A601B7018C899D89A0E069
:1001C0000E94FF2E09F00DC1AD80BE80CF80D88483
:1001D000E984FA840B851C8520E033E245E75EEE76
:1001E00064E170E080E090E00E94472EC901DA01EE
:1001F000A901BD0120FF99C04F5F5F4F6F4F7F4F37
:1002000049835A836B837C834F3F51056105710598
:1002100040F08EEF90E0A0E0B0E089839A83AB835A
:10022000BC83E980FA800B811C81A8019701AD8015
:10023000BE80CF80D884E984FA840B851C8560E079
:1002400070E080E090E00E94912D29013A014B017D
:100250001C01211504E030070BE6400704EF5007AE
:1002600004E1600771058105910509F008F47DC07E
:1002700089819A81AB81BC810297A109B1098983E7
:100280009A83AB83BC831C012D010B859101A201D4
:1002900060E070E080E090E00E94912D29013A0139
:1002A0004B011C0189819A81AB81BC819927AA27C6
:1002B000BB27ED85FE8580839183A283B38314825F
:1002C0001582168217821086118612861386920175
:1002D000A301B401C10165960FB6F894DEBF0FBE4D
:1002E000CDBFDF91CF911F910F91FF90EF90DF90E5
:1002F000CF90BF90AF909F908F907F906F905F90C6
:100300004F903F902F90089545E050E060E070E0FE
:100310001D8286ED8E8391E19F83AEE7A887B3E0CF
:10032000B9871A861B861C8667CF0597A105B1057C
:1003300009F066CF16E0E12EF12C00E010E0E98232
:10034000FA820B831C836DCF46E057E060E070E0DB
:10035000E0E8ED83F0EFFE830AEF0F8312E01887E9
:1003600019861A861B861C864BCF2F3F3F484F426B
:100370005045694071058105910511F008F092CF53
:1003800089819A81AB81BC810296A11DB11D8983AF
:100390009A83AB83BC831C012D01AD80BE80CF80CE
:1003A000D884E984FA840B851C8570CF412C63C006
:1003B00029813F85488959896A897B898C899D89EA
:1003C000A0E00E94FF2E09F49FCF1D82B6EDBE83F0
:1003D000E1E1EF83FEE7F88703E009871A861B86D1
:1003E0001C86AD80BE80CF80D884E984FA840B85DA
:1003F0001C8529813F85488959896A897B898C892F
:100400009D890E94452E29013A014B011C01A0E063
:100410000E94FF2E59F629813F85488959896A89AA
:100420007B898C899D890E94472E022F132F242FB0
:10043000352FD901C8010697A109B109893F910556
:10044000A105B10508F043CF10E030E020E0AD8514
:10045000BE850D931D932D933C931397FD0114823C
:1004600015821682178218961D921D921D921C925B
:100470001B9744244394512C612C712C812C912C7A
:10048000212C312C24CF29813F85488959896A89BB
:100490007B898C899D89A0E00E94FF2E09F454CFAE
:1004A00010E81D8380EF8E839AEF9F83A2E0A887D8
:1004B000198694CFDF92EF92FF920F931F93CF9301
:1004C000DF93FC01E080F18002811381D481C5813A
:1004D000B681D7809701A8016D2F7C2F8B2F9D2D82
:1004E0002C5D354C4241510961097109810991091D
:1004F0002B3D354C42415105610571058105910542
:1005000009F0D0F49701A8016D2F7C2F8B2F9D2D22
:1005100007E00E94B42E2083318342835383648397
:1005200075838683978387E0DF91CF911F910F9129
:10053000FF90EF90DF9008959701A8016D2F7C2F19
:100540008B2F9D2D285B3B4845425109610971095C
:1005500081099109273B3B484542510561057105D9
:100560008105910509F098F49701A8016D2F7C2F62
:100570008B2F9D2D06E00E94B42E20833183428371
:100580005383648375838683978386E0CDCF9701F9
:10059000A8016D2F7C2F8B2F9D2D205737414B4469
:1005A000510961097109810991092F3637414B447D
:1005B0005105610571058105910509F098F49701D0
:1005C000A8016D2F7C2F8B2F9D2D05E00E94B42E4E
:1005D0002083318342835383648375838683978327
:1005E00085E0A2CF9701A8016D2F7C2F8B2F9D2D29
:1005F000205E3E424649510961097109810991090C
:100600002F3D3E4246495105610571058105910521
:1006100009F098F49701A8016D2F7C2F8B2F9D2D49
:1006200004E00E94B42E2083318342835383648389
:1006300075838683978384E077CF9701A8016D2F18
:100640007C2F8B2F9D2D205C3D454C4251406109F4
:100650007109810991092F3B3D454C42514061058B
:1006600071058105910509F098F49701A8016D2F96
:100670007C2F8B2F9D2D03E00E94B42E208331838D
:1006800042835383648375838683978383E04CCF4F
:100690009701A8016D2F7C2F8B2F9D2D20583B4B50
:1006A0004845524061097109810991092F373B4B37
:1006B00048455240610571058105910509F098F49E
:1006C0009701A8016D2F7C2F8B2F9D2D02E00E949A
:1006D000B42E20833183428353836483758386835E
:1006E000978382E021CF9701A8016D2F7C2F8B2F5C
:1006F0009D2D3757414B544061097109810991097A
:100700002F3F3647414B54406105710581059105E6
:1007100009F098F49701A8016D2F7C2F8B2F9D2D48
:1007200001E00E94B42E208331834283538364838B
:1007300075838683978381E0F7CE80E0F5CE2F9294
:100740003F924F925F926F927F928F929F92AF9261
:10075000BF92CF92DF92EF92FF920F931F93CF93AE
:10076000DF93CDB7DEB76C970FB6F894DEBF0FBE40
:10077000CDBF322E3D87242E5E872B013C01A982FE
:10078000BF86C88AD98AEA8AFB8A0C8B1D8B988E11
:100790008F8A211501EC30070AE140070DE350076D
:1007A00005E0600771058105910509F0A0F52F3777
:1007B00010EF31071AEF410712E05107610571058B
:1007C0008105910509F008F4B4C12F3F354D414131
:1007D0005E47634071058105910509F008F48FC0FB
:1007E00029813F85488959896A897B898C899D89B6
:1007F000A0E0992493940E94FF2E09F08EC011E08E
:100800001E8B94E0892E912CA12CB12C89869A867E
:10081000AB86BC862FC0312CB1ECBD872AE1222EDD
:10082000EDE3EE8735E0432E512C612C712CD8CFAF
:10083000A32CBD84C22CDE847201830120E034E04D
:100840004BE654EF64E170E080E090E00E94472EB8
:10085000122FB32FF42FE52FA7E00E94FF2E21F4D3
:1008600016E0B0E0F0E0E0E0CF011987BA879B879F
:10087000EC871E8A89849A84AB84BC84A501940188
:1008800060E070E0CB01A32CBD84C22CDE84720139
:10089000830129833A834B835C836D837E838F83BB
:1008A000988760E070E080E090E00E94912D2983BD
:1008B0003F87488B598B6A8B7B8B8C8B9D8B0E89EA
:1008C000C12CD12C7601C39440E050E0BA01013034
:1008D00009F0A9C0AF89B88D1D921D921D921C927E
:1008E0001397FD01148215821682178281E090E031
:1008F000A0E0B0E080879187A287B387DEC029811E
:100900003F85488959896A897B898C899D89A0E0BE
:100910000E94FF2E09F48CCF912CA32CBD84C22CF5
:10092000DE847201830129813F85488959896A895A
:100930007B898C899D890E94472E29873A874B871E
:100940005C8729853A854B855C8506E0A02EB12C15
:10095000263031054105510568F089859A85AB85BA
:10096000BC8589309740A105B105D0F0B8E0AB2E29
:1009700017E0B12EC12CD12CE12CF12C00E010E0BD
:1009800029813F85488959896A897B898C899D8914
:100990000E94472E322E3D87242E5E872B013C017C
:1009A000A32CBD84C22CDE847201830129813F8582
:1009B000488959896A897B898C899D890E94452E3D
:1009C000E0E4AE2EF2E4BF2EAFE0CA2ED12CE12C33
:1009D000F12C00E010E00E94912DA32CBD84C22CCC
:1009E000DE84720183010E94472EA32FF42FE52F8E
:1009F000422F5A2F6F2F7E2FA0E4CA2EA2E4DA2EA8
:100A0000AFE0EA2EF12C411551056105710521F485
:100A1000C12CD12C7601C394AA24A3949A1409F46E
:100A20006DC001E00E8BCB01BA0117E0660F771F96
:100A3000881F991F1A95D1F7A70196010E94692D69
:100A4000298F3A8F4B8F5C8F89849A84AB84BC84C6
:100A500007E0880C991CAA1CBB1C0A95D1F79501CC
:100A6000840112502109310948015901298D3A8D1B
:100A70004B8D5C8D280D391D4A1D5B1DAF89B88DCE
:100A80002D933D934D935C931397FD016483758380
:100A9000868397831896CD92DD92ED92FC921B97F8
:100AA0008E88882051F039829D849F86288AAE8462
:100AB000A98A4A8A5B8A6C8A7D8A29813F8548890E
:100AC00059896A897B898C899D896C960FB6F894BF
:100AD000DEBF0FBECDBFDF91CF911F910F91FF9071
:100AE000EF90DF90CF90BF90AF909F908F907F90CE
:100AF0006F905F904F903F902F900895AF89B88D81
:100B00001D921D921D921C921397FD011482158255
:100B10001682178281E090E0A0E0B0E080879187A4
:100B2000A287B3873982FD85FF87288A8E84898AC8
:100B3000C0CF29813F85488959896A897B898C89F9
:100B40009D89A0E0E0E83E2EF0EFFD87FAEF2F2E22
:100B500002E00E87412C512C612C712C0E94FF2E3B
:100B600009F0DACE18E0B7E07DCEDF92EF92FF9287
:100B70000F931F93CF93DF93FC01E080F1800281FC
:100B80001381D481C581B681D7809701A8016D2FCB
:100B90007C2F8B2F9D2D20583A41464051096109E9
:100BA0007109810991092F373A4146405105610584
:100BB00071058105910509F0D0F49701A8016D2F09
:100BC0007C2F8B2F9D2D07E00E94B42E2083318334
:100BD00042835383648375838683978387E0DF91A1
:100BE000CF911F910F91FF90EF90DF9008959701A3
:100BF000A8016D2F7C2F8B2F9D2D35534C40510913
:100C000061097109810991092F3F34434C40510515
:100C1000610571058105910509F098F49701A80116
:100C20006D2F7C2F8B2F9D2D06E00E94B42E2083EC
:100C3000318342835383648375838683978386E0FD
:100C4000CECF9701A8016D2F7C2F8B2F9D2D3A566B
:100C50004841510961097109810991092F3F3946BC
:100C600048415105610571058105910509F098F428
:100C70009701A8016D2F7C2F8B2F9D2D05E00E94E1
:100C8000B42E2083318342835383648375838683A8
:100C9000978385E0A4CF9701A8016D2F7C2F8B2F20
:100CA0009D2D345D40435109610971098109910904
:100CB0002F3F334D40435105610571058105910575
:100CC00009F098F49701A8016D2F7C2F8B2F9D2D93
:100CD00004E00E94B42E20833183428353836483D3
:100CE00075838683978384E07ACF9701A8016D2F5F
:100CF0007C2F8B2F9D2D385A41465109610971096E
:100D0000810991092F3F374A414651056105710517
:100D10008105910509F098F49701A8016D2F7C2FAA
:100D20008B2F9D2D03E00E94B42E208331834283BC
:100D30005383648375838683978383E050CF9701C1
:100D4000A8016D2F7C2F8B2F9D2D3055434C5109C1
:100D500061097109810991092F3F3F44434C5105B5
:100D6000610571058105910509F098F49701A801C5
:100D70006D2F7C2F8B2F9D2D02E00E94B42E20839F
:100D8000318342835383648375838683978382E0B0
:100D900026CF9701A8016D2F7C2F8B2F9D2D305AC8
:100DA0004648514061097109810991092F3F3F4926
:100DB00046485140610571058105910509F098F497
:100DC0009701A8016D2F7C2F8B2F9D2D01E00E9494
:100DD000B42E208331834283538364837583868357
:100DE000978381E0FCCE80E0FACE089508950895BF
:100DF000AF92BF92CF92DF92EF92FF920F931F9329
:100E0000CF93DF936C017B018B01040F151FEB0166
:100E10005E01AE18BF08C017D10759F06991D6011D
:100E2000ED91FC910190F081E02DC6010995892B8F
:100E300079F7C501DF91CF911F910F91FF90EF904E
:100E4000DF90CF90BF90AF900895FC014481558111
:100E5000608171818CEA95E00C94F806FC01538D59
:100E6000448D252F30E0842F90E0821B930B541784
:100E700010F0CF96089501970895FC01918D828D11
:100E8000981761F0A28DAE0FBF2FB11D5D968C91AA
:100E9000928D9F5F9F73928F90E008958FEF9FEFE9
:100EA0000895FC01918D828D981731F0828DE80FA5
:100EB000F11D858D90E008958FEF9FEF0895FC015F
:100EC000918D228D892F90E0805C9F4F821B91092C
:100ED0008F739927089587E694E00E945F0721E0C9
:100EE000892B09F420E0822F089580E090E0892B7F
:100EF00029F00E946B0781110C9400000895FC01F9
:100F0000A48DA80FB92FB11DA35ABF4F2C91848D6A
:100F100090E001968F739927848FA689B7892C93C7
:100F2000A089B1898C91837080648C93938D848D1A
:100F3000981306C00288F389E02D80818F7D80831D
:100F40000895EF92FF920F931F93CF93DF93EC01DD
:100F500081E0888F9B8D8C8D98131AC0E889F98960
:100F6000808185FF15C09FB7F894EE89FF89608363
:100F7000E889F98980818370806480839FBF81E0E4
:100F800090E0DF91CF911F910F91FF90EF90089526
:100F9000F62E0B8D10E00F5F1F4F0F731127E02E01
:100FA0008C8D8E110CC00FB607FCFACFE889F98939
:100FB000808185FFF5CFCE010E947F07F1CFEB8DB9
:100FC000EC0FFD2FF11DE35AFF4FF0829FB7F8940D
:100FD0000B8FEA89FB8980818062CFCFCF93DF932B
:100FE000EC01888D8823B9F0AA89BB89E889F98941
:100FF0008C9185FD03C0808186FD0DC00FB607FC76
:10100000F7CF8C9185FFF2CF808185FFEDCFCE01A8
:101010000E947F07E9CFDF91CF910895833081F05F
:1010200028F4813099F08230A9F008958730A9F032
:101030008830C9F08430B1F4809180008F7D03C086
:10104000809180008F7780938000089584B58F779A
:1010500084BD089584B58F7DFBCF8091B0008F77DC
:101060008093B00008958091B0008F7DF9CFCF9329
:10107000DF93282F30E0F901E255FF4F8491F90109
:10108000E656FF4FD491F901EA57FF4FC491CC23A4
:10109000A1F081110E940E08EC2FF0E0EE0FFF1F6F
:1010A000E458FF4FA591B491EC91ED2381E090E0DD
:1010B00009F480E0DF91CF91089580E090E0FACFCD
:1010C0001F93CF93DF93282F30E0F901E255FF4FB4
:1010D0008491F901E656FF4FD491F901EA57FF4F89
:1010E000C491CC23A9F0162F81110E940E08EC2F79
:1010F000F0E0EE0FFF1FEE58FF4FA591B4918FB7B0
:10110000F894EC91111108C0D095DE23DC938FBFC9
:10111000DF91CF911F910895DE2BF8CFCF93DF930E
:1011200090E0FC01E656FF4F24918A579F4FFC0147
:1011300084918823C9F090E0880F991FFC01E85939
:10114000FF4FA591B491FC01EE58FF4FC591D4918A
:1011500061110DC09FB7F8948C91209582238C93D8
:101160008881282328839FBFDF91CF910895623023
:1011700051F49FB7F8943C91822F809583238C93F0
:10118000E8812E2BEFCF8FB7F894EC912E2B2C9378
:101190008FBFEACF3FB7F8948091E5039091E603C3
:1011A000A091E703B091E80326B5A89B05C02F3FA7
:1011B00019F00196A11DB11D3FBFBA2FA92F982F7D
:1011C0008827BC01CD01620F711D811D911D42E078
:1011D000660F771F881F991F4A95D1F708958F9240
:1011E0009F92AF92BF92CF92DF92EF92FF924B010C
:1011F0005C010E94CA086B017C010E94CA086C193C
:101200007D098E099F09683E734081059105A8F309
:1012100021E0821A9108A108B10888EEC80E83E087
:10122000D81EE11CF11C81149104A104B10429F71A
:10123000FF90EF90DF90CF90BF90AF909F908F90F6
:1012400008952091C103260F3327331F2132310522
:10125000ECF420913D04FC0190E080E0243069F042
:1012600082E00895A091C1032191AC014F555C4FDC
:10127000A40FB52FB11D2C930196861798F380917A
:10128000C103680F6093C10380E0089581E0089571
:1012900010923D0481E080933C041092170461E0B9
:1012A00082E10E94600861E083E10E946008E9EB4E
:1012B000F0E080818E7F808380818D7F808388E4D1
:1012C0008093B80085E48093BC000895CF93DF93AA
:1012D00091E09093A0038823B9F0C091B800D09119
:1012E000BA008091BC008A7B8093BC0060E082E100
:1012F0000E94600860E083E10E9460080E94480943
:10130000D093BA00C093B800DF91CF9108958F9227
:101310009F92AF92BF92CF92DF92EF92FF920F9384
:101320001F93CF93DF93D0916604D13208F0D7C0DA
:10133000182FC09165040E94CA086B017C0180913E
:101340003D0481116BC082E080933D0410933C0406
:101350008FEF80933B0410923A04D0933904A5E4B4
:10136000B4E0E9E1F4E080E0D81391C010921804F1
:1013700080911804CC0FC82BC093180480911704D7
:10138000813009F088C0109217040E94CA086B01CE
:101390007C01809118048093BB0080913F04909160
:1013A0004004A0914104B0914204892B8A2B8B2BDD
:1013B000A1F00E94CA0800913F04109140042091BE
:1013C0004104309142046C197D098E099F0906176A
:1013D00017072807390708F442C08091BC0083FD35
:1013E000D8CF85EC8093BC000E94CA086B017C01B9
:1013F00080913D04823009F450C080913B048F3FBE
:1014000009F46FC080913B04803209F46CC0809174
:101410003B04803309F469C084E026C080913F0416
:1014200090914004A0914104B0914204892B8A2BF1
:101430008B2B09F484CF0E94CA0880903F049090BF
:101440004004A0904104B09042046C197D098E09BB
:101450009F0986169706A806B90608F070CF8091F6
:101460003E040E94660985E01092440410926604CE
:1014700010924304DF91CF911F910F91FF90EF9055
:10148000DF90CF90BF90AF909F908F9008959D91E7
:1014900091938F5F69CF85EEA5CF80913F049091A6
:1014A0004004A0914104B0914204892B8A2B8B2BDC
:1014B00009F49ECF0E94CA0800913F041091400495
:1014C00020914104309142046C197D098E099F09D5
:1014D000061717072807390708F08ACFC0CF81E021
:1014E000C3CF80E0C1CF82E0BFCF83E0BDCF0895FE
:1014F000E091F6038091F503E81730F4F0E0E9504D
:10150000FC4F808190E008958FEF9FEF08959091B8
:10151000F6038091F5032FEF3FEF981748F4E92F7A
:10152000F0E0E950FC4F208130E09F5F9093F6039C
:10153000C9010895CF92DF92EF92FF920F931F930C
:10154000CF93DF937C01CB018A01209143042223B6
:1015500089F0EB016B01C40ED51ECC15DD0569F0D9
:101560006991D701ED91FC910190F081E02DC701C7
:101570000995F3CF642F0E942109C801DF91CF9113
:101580001F910F91FF90EF90DF90CF900895CF9330
:10159000DF931F92CDB7DEB76983209143042223E6
:1015A000F9F020916604203258F021E030E0FC018F
:1015B0003383228390E080E00F90DF91CF910895F4
:1015C00080914404E82FF0E0EB5BFB4F998190831E
:1015D0008F5F809344048093660481E090E0ECCFB9
:1015E00061E0CE0101960E942109F7CFCF93C62F6B
:1015F0009091AB0521E020934304909365041092F1
:10160000440410926604682F84E095E00E94C70AA3
:101610006C2F84E095E00E94C70A81E0CF910C9482
:10162000870960E2009719F0019721F460E881EBE7
:101630000C94F60A0895EF92FF920F931F93CF93A5
:10164000DF93062F7A019091AB0521E020934304AC
:10165000909365041092440410926604682F84E00D
:1016600095E00E94C70AE70110E0CE018E199F099C
:101670008017910734F4699184E095E00E94C70ACD
:10168000F4CF81E0DF91CF911F910F91FF90EF9008
:101690000C94870990E080E008958BE00E94370861
:1016A000892B89F564E170E080E090E00E94EF080A
:1016B0008BE00E943708892B31F58BE00E943708B8
:1016C000892BD9F3E0910601F09107013197E930B8
:1016D000F105C8F4E259F44F0C948B2D770B840B71
:1016E000890B8E0B930B980B9D0BA20BA70B81E024
:1016F00090E0A0E0B0E08093020190930301A093FA
:101700000401B093050108958AE090E0A0E0B0E004
:10171000F2CF84E690E0A0E0B0E0EDCF88EE93E079
:10172000A0E0B0E0E8CF80E197E2A0E0B0E0E3CF56
:1017300080EA96E8A1E0B0E0DECF80E492E4AFE09A
:10174000B0E0D9CF80E896E9A8E9B0E0D4CF80E056
:1017500091EEA5EFB5E0CFCFCF92DF92EF92FF925F
:101760000F931F93CF93DF939091AB0521E02093CC
:101770004304909365041092440410926604682F09
:1017800084E095E00E94C70A81E00E948709C09129
:10179000AB050E94CA086B017C0180913D04811158
:1017A00065C081E080933D0410923C049FEF9093CC
:1017B0003B0410923A0410923904809318048091EB
:1017C0001804CC0FC82BC0931804809117048130E3
:1017D00009F080C0109217040E94CA086B017C01B6
:1017E000809118048093BB0080913F049091400445
:1017F000A0914104B0914204892B8A2B8B2BA1F03C
:101800000E94CA0800913F041091400420914104B5
:10181000309142046C197D098E099F09061717073C
:101820002807390708F443C08091BC0083FDD8CF56
:1018300085EC8093BC000E94CA086B017C018091FA
:101840003D04813009F448C080913A04C1E081111F
:1018500002C0C0913A04E9E1F4E0A7EFB3E080E010
:101860008C1751F191919D938F5FFACF80913F0436
:1018700090914004A0914104B0914204892B8A2B9D
:101880008B2B09F48ACF0E94CA0800913F04109163
:10189000400420914104309142046C197D098E0965
:1018A0009F09061717072807390708F076CF809198
:1018B0003E040E946609C0E01092F603C093F5034F
:1018C0008091F603C81751F184E095E00E94870AE1
:1018D000D82FF6CF85EEADCF80913F049091400494
:1018E000A0914104B0914204892B8A2B8B2B09F4DF
:1018F000A6CF0E94CA0800913F0410914004209195
:101900004104309142046C197D098E099F09061724
:1019100017072807390708F092CFC9CF8D2FDF911D
:10192000CF911F910F91FF90EF90DF90CF9008958E
:101930001F93CF93DF93D62F142FC4E483309105E8
:1019400089F048F4C4E38130910561F0CCE302975B
:1019500049F0CCE207C0CCE48430910519F0C4E52D
:101960000597B9F78C2F0E94AC0B837811118C600E
:1019700090E1D99FB0011124682B8C2FDF91CF917A
:101980001F910C94F60ACF93DF93D62FC0E1C80FB6
:101990008C2F0E94AC0B682FD13031F460648C2FF7
:1019A000DF91CF910C94F60A6F7BF9CFCF93DF9341
:1019B000D82FC62F83E00E94AC0B61E070E001C01D
:1019C000660FDA95EAF7C13039F46095682383E051
:1019D000DF91CF910C94F60A682BF9CFFF920F9309
:1019E0001F93CF93DF93EC018B01F82E80E1F80E6B
:1019F0008F2D0E94AC0B682F0115110581F46F7DAE
:101A00008F2D0E94F60ACC0FDD1FC65CDA4F1A87B5
:101A10000987DF91CF911F910F91FF900895606228
:101A2000EFCFCF93DF93EC0160E08E810E946008DE
:101A300061E08E810E94600860E08E810E946008F3
:101A40008BE891E00197F1F7DF91CF910895CF9264
:101A5000DF92EF92FF920F931F93CF93DF936C016E
:101A60008C01095F1F4FD0E0C0E0E62EF12C61E051
:101A7000F80181918F010E948E08B7010C2E02C0DF
:101A8000759567950A94E2F76170F8013197808146
:101A90000E9460082196C430D10549F7C601DF9144
:101AA000CF911F910F91FF90EF90DF90CF900C940A
:101AB000110DCF92DF92EF92FF920F931F93CF936E
:101AC000DF93EC01F62E642F8C810E9460088D81DB
:101AD0008F3F19F060E00E9460080F2D10E08F85A5
:101AE00084FF2BC06E0187E0C80ED11CF12CE12CC5
:101AF00061E0F60181916F010E948E08B8010E2C01
:101B000002C0759567950A94E2F76170F601319706
:101B100080810E946008FFEFEF1AFF0A88E0E81654
:101B2000F10431F7CE01DF91CF911F910F91FF901A
:101B3000EF90DF90CF900C94110DB80184E0759573
:101B400067958A95E1F7CE010E94270D6F2DCE0192
:101B5000DF91CF911F910F91FF90EF90DF90CF9089
:101B60000C94270D40E0682F8CEA95E00C94590DF9
:101B70009091BF05691710F06FEF690FE62FF0E045
:101B8000E455FA4F9489890F80680C94B20D81E076
:101B90000E94B20D8BE39FE10197F1F70895CF9377
:101BA000DF93823029F49091BB0598609093BB0538
:101BB0008093BF051092C00580E48093C10580E149
:101BC0008093C20580E58093C3058BE39DE0019778
:101BD000F1F760E08091B0050E94600860E08091BC
:101BE000B2050E9460088091B1058F3F19F060E056
:101BF0000E9460088091BB0584FD34C063E08CEADC
:101C000095E00E94270DCBE4D6E4CE010197F1F7D1
:101C100063E08CEA95E00E94270D2197F1F763E0DD
:101C20008CEA95E00E94270D83E592E00197F1F799
:101C300062E08CEA95E00E94270D8091BB058062EE
:101C40000E94B20D84E08093BC058CE00E94B20D2E
:101C50000E94C70D82E08093BD0586E0DF91CF91A1
:101C60000C94B20D80620E94B20D8BE496E4019751
:101C7000F1F78091BB0580620E94B20D83E592E08E
:101C80000197F1F78091BB0580620E94B20DD5CF1C
:101C90000F931F93CF93DF938C018BE00E94370843
:101CA000892B09F069C0C0910001D091010160E069
:101CB0008CE08C1B0E94B80D01301105C1F52196F6
:101CC000C830D10571F1CC30D10571F1C430D105E6
:101CD00009F1D0930101C0930001209100013091DE
:101CE000010124303105E4F530930701209306010A
:101CF00060E08CE0821B0E94B80D8091BC05982F9B
:101D000092609093BC058A60DF91CF911F910F91F3
:101D10000C94B20D85E090E0909301018093000156
:101D2000DCCF89E090E0F8CF8BE090E0F5CF0F3F7B
:101D30001F4F99F680910001909101010197843025
:101D4000910541F08830910541F0009729F781E035
:101D500090E0E2CF83E090E0DFCF87E090E0DCCF5F
:101D6000C9012830310534F401979093070180931D
:101D70000601BECF0297F9CF8091BC058D7F80937D
:101D8000BC0588600E94B20D0130110521F540911B
:101D9000020150910301609104017091050180914D
:101DA000320190913301A0913401B0913501840F3B
:101DB000951FA61FB71F8093320190933301A09304
:101DC0003401B093350181E080934401DF91CF91DC
:101DD0001F910F9108950F3F1F4FA9F78091320176
:101DE00090913301A0913401B091350140910201ED
:101DF0005091030160910401709105014817590742
:101E00006A077B0700F7409102015091030160913E
:101E1000040170910501841B950BA60BB70BCBCF6A
:101E200041E00E94590D81E090E008950F931F93C7
:101E3000CF93DF938B0128E0829FC001112480643F
:101E40000E94B20DE801085F1F4F69918CEA95E08E
:101E50000E94100FC017D107C1F7DF91CF911F91DA
:101E60000F91089541E0682F8CEA95E00E94590D8A
:101E700081E090E0089520912F0530913005232BCB
:101E800039F421E0FC018081882361F020E00AC060
:101E9000BC0180912B0590912C050E94F63021E029
:101EA000892BA1F7822F08958F929F92AF92BF92B4
:101EB0000F931F93CF93DF93CDB7DEB7A1970FB6E4
:101EC000F894DEBF0FBECDBF19A2423008F44AE03D
:101ED0008E010F5D1F4F842E912CB12CA12CA501DA
:101EE00094010E94692DE62FB901CA01EA3044F538
:101EF000E05DD801EE938D01232B242B252B79F760
:101F000090E080E0109769F0FD0101900020E9F772
:101F10003197AF014A1B5B0BBD018CEA95E00E9433
:101F2000F806A1960FB6F894DEBF0FBECDBFDF91C5
:101F3000CF911F910F91BF90AF909F908F90089578
:101F4000E95CD7CFFC0101900020E9F73197AF01A0
:101F5000481B590BBC018CEA95E00C94F806CF9213
:101F6000DF92EF92FF92CF93DF9360E081E00E94D7
:101F7000B80D6091320170913301809134019091DC
:101F8000350120E432E44FE050E00E94692D690100
:101F90007A01E9012436310540F480E20E94320FD3
:101FA0002A9718F480E20E94320F4AE0C701B60176
:101FB0000E94540F8EE20E94320F609132017091A4
:101FC0003301809134019091350120E432E44FE0F7
:101FD00050E00E94692D28EE33E040E050E00E947E
:101FE000692D69017A01E9012436310540F480E365
:101FF0000E94320F2A9718F480E30E94320F4AE0C1
:10200000C701B6010E94540F8EE20E94320F609108
:10201000320170913301809134019091350128EEA5
:1020200033E040E050E00E94692D6B017C01EB0140
:102030006436710540F480E30E94320F2A9718F449
:1020400080E30E94320F4AE0C701B6010E94540F9C
:102050008DE692E00E94A20F61E080E00E94B80D40
:102060008BE295E00E94250781EA91E0DF91CF9114
:10207000FF90EF90DF90CF900C94A20FCF93DF935F
:10208000EC0180911A0590911B050097E9F0688199
:10209000798161157105B1F040911C0550911D05C4
:1020A0002C813D814217530768F00E94FF308C81DC
:1020B0009D8190931F0580931E051D821C82DF91D8
:1020C000CF9108950E94A72F8881998190931B0535
:1020D00080931A058A819B8190931D0580931C052E
:1020E0008C819D8190931F0580931E051982188213
:1020F0001B821A82E2CFFC0180819181009711F04E
:102100000C94A72F08952F923F924F925F926F9257
:102110007F928F929F92AF92BF92CF92DF92EF9277
:10212000FF920F931F93CF93DF93CDB7DEB72D9719
:102130000FB6F894DEBF0FBECDBF3C01C982DA8274
:10214000EB82FC820D831E832F83388749875A8751
:102150006B877C87BAA03C2C2D2C5E2C0D87412EE2
:10216000922EC984DA84EB84FC8484E190E00E949E
:102170000B2F8C01FC01D082C182862D880F880F25
:10218000880F845D0E94AC0BF52DF3705F2E8C7F61
:10219000582AF8015282238234828CE0F694E79424
:1021A000D794C7948A95D1F7FC2DF07FCF2E892D37
:1021B0008F70C82AF801C58246828D85878393E097
:1021C0006916710409F46CC0A8F5F1E06F1671048A
:1021D00009F448C082E06816710409F452C0A801ED
:1021E00068E08AE20E941B0B6A2D90E080E00E946A
:1021F000C30C4B2D682D90E080E00E94980CC80124
:102200002D960FB6F894DEBF0FBECDBFDF91CF91F4
:102210001F910F91FF90EF90DF90CF90BF90AF9004
:102220009F908F907F906F905F904F903F902F90F6
:102230000C94A72F94E06916710409F440C0E5E0FE
:102240006E16710461F6A80168E082E50E941B0B1E
:102250006A2D85E090E00E94C30C4B2D682D85E02F
:1022600090E0CBCFA80168E082E30E941B0B6A2DAF
:1022700081E090E00E94C30C4B2D682D81E090E03E
:10228000BCCFA80168E08AE30E941B0B6A2D82E0A4
:1022900090E00E94C30C4B2D682D82E090E0ADCF02
:1022A000A80168E082E40E941B0B6A2D83E090E0A5
:1022B0000E94C30C4B2D682D83E090E09ECFA801B7
:1022C00068E08AE40E941B0B6A2D84E090E00E9483
:1022D000C30C4B2D682D84E090E08FCF2F923F925E
:1022E0004F925F926F927F928F929F92AF92BF9226
:1022F000CF92DF92EF92FF920F931F93CF93DF93D2
:10230000CDB7DEB76D970FB6F894DEBF0FBECDBF69
:102310002A8B3B8B4C8B5D8B6E8B7F8B888F998F41
:102320001B8F0A8F6091A3057091A4058091A5056C
:102330009091A60524E630E040E050E00E94E92DAF
:10234000522E632E742E852E962E7E878D87492ED3
:102350008091A7059091A805A091A905B091AA0523
:102360006C017D01FF0CCC08DC2C76019C01AD01D9
:102370006C2D7C2D8C2D9C2D0FE10E94B42EA12C58
:10238000EAECBE2EFAE9CF2EABE3DA2EE12CF12CEB
:1023900000E010E00E94162EA52CB62CC72CD82CDD
:1023A000E92CFE840D85142D0E94912D0FE10E94D1
:1023B000CF2E29833A834B835C836D837E838F8307
:1023C000988789819A81AB81BC81BB0F880B982F3C
:1023D000DC0189879A87AB87BC87252D362D472D51
:1023E000582D692D7F2D8D85942DA980BA80CB80A5
:1023F000DC80E984FE2C0E2D1E2D0E94EA2E190190
:1024000049875D876E877F87888B998B6A887B88F1
:102410008C889D889E899D8FAF89AC8F488C598C04
:102420009301A401692F7A2FC201211534404B4634
:10243000544F644171058105910569F060F0612C8C
:1024400044E0742E5BE6852E64EF962EE4E1ED8F7A
:102450001C8E412C512C9301A4016D8D7C8DC201E9
:10246000211530494F42504569407105810591055C
:1024700060F4612C90E9792E2FE2822E30E5932EC4
:1024800089E08D8F1C8E412C512C5101C984DD8433
:10249000EE84FF84088919899301A4016D8D7C8DD8
:1024A000C2010E94472E29833A834B835C83898132
:1024B0009A81AB81BC810F97A105B10508F0D2C00C
:1024C0008FE0A82EB12CC12CD12CE12CF12C00E0F6
:1024D00010E0910149855D856E857F8588899989A0
:1024E0000E94912D39014A016D8F7C8F2C01510181
:1024F000C984DD84EE84FF84088919899301A401CD
:102500006D8D7C8DC2010E94452EA0E4AA2EB2E4FE
:10251000BB2E1FE0C12ED12CE12CF12C00E010E0ED
:102520000E94912D5101C984DD84EE84FF840889C5
:1025300019890E94472EC901DA01812C912C54017E
:1025400083940097A105B10539F0E0E48E2EE2E412
:102550009E2EEFE0AE2EB12CBC01CD0127E0660F20
:10256000771F881F991F2A95D1F7A50194010E9412
:10257000692D362E272E182F49805A806B807C803B
:1025800067E0440C551C661C771C6A95D1F792E0F5
:10259000591A61087108420E531E641E751E84E1AB
:1025A00090E00E940B2F9A838983DC019C92119604
:1025B0008C921197862D837012968C931297139696
:1025C0005C92139714964C927CE0B694A7949794DF
:1025D00087947A95D1F7B82DB07F8B2E812AE98127
:1025E000FA818582268237828A8D9B8D892B09F01C
:1025F00046C0AF0168E08AE10E941B0B9A89909364
:102600009305AB89A0939405BC89B0939505ED899A
:10261000E0939605FE89F09397058F89809398053E
:10262000988D90939905A98DA0939A0589819A8197
:102630006D960FB6F894DEBF0FBECDBFDF91CF9180
:102640001F910F91FF90EF90DF90CF90BF90AF90D0
:102650009F908F907F906F905F904F903F902F90C2
:102660000C94A72F89819A81AB81BC818B35910510
:10267000A105B10508F43BCF0AE5A02E23CFEA8DD2
:10268000FB8D319799F649815A8168E082E20E9478
:102690001B0BFA89F0939B058B8980939C059C8981
:1026A00090939D05AD89A0939E05BE89B0939F052B
:1026B000EF89E093A005F88DF093A105898D8093B3
:1026C000A205B4CF2F923F924F925F926F927F926A
:1026D0008F929F92AF92BF92CF92DF92EF92FF9232
:1026E0000F931F93CF93DF93CDB7DEB7E5970FB668
:1026F000F894DEBF0FBECDBFE22E29A3F32E3AA37E
:102700004BA35CA36DA37EA38FA398A7702E612E0D
:102710009701AFEF0E94F32E2E373A414640510504
:10272000610571058105910509F058F480E889A3D8
:102730008AE18AA386E08BA31CA21DA21EA21FA26F
:1027400018A629A13AA14BA15CA16DA17EA18FA1E0
:1027500098A52115314C4A415D43654071058105BD
:10276000910569F060F019A281EC8AA38AE18BA33C
:102770008DE38CA385E08DA31EA21FA218A6D9A06D
:102780004AA05BA0ACA0EDA0FEA00FA118A5272C2D
:10279000362C2D2D342D452D5A2DB701C80121156C
:1027A000344E4B405445624071058105910509F056
:1027B00008F42CC1A3E54A2EA5E05A2E2AE335E001
:1027C0003AA729A78901F201D12CC101880F991FCD
:1027D000DC01AD5BBA4F7D012081318142815381A3
:1027E000648175818681978138962115344E4B40DE
:1027F0005445624071058105910571F068F0D71468
:1028000059F0D80119962D913C91D7018D919C9149
:102810002817390709F46FC1D3940E5F1F4FB6E034
:10282000DB12DACF61E0872D962D0E94D60C29A10C
:102830003AA14BA15CA16DA17EA18FA198A5D10168
:10284000E3E0AA0FBB1FEA95E1F7A65CBA4FFD01D2
:10285000799659962C93318342835383648375838D
:1028600086839783FE013D964F01A12CB12CC12C8C
:10287000D12CE12CF12C00E010E00E949F032BA74B
:102880003CA74DA75EA76FA778AB89AB9AABC101F8
:10289000880F991F9C01265C3A4F7901D90119963E
:1028A0000D911C912BA53CA589A99AA90E946E1196
:1028B000712C612CF7013996FDABECABD201AC90D9
:1028C0001196EC9011971296FC90129713960C911A
:1028D000139714961C9114971596BC91F201D6800B
:1028E000C780F8E04F0E511C2A2D3E2D4F2D502F42
:1028F000612F7B2F8D2D9C2DA0E00E94FF2E09F4CF
:1029000055C0E9A5FAA521853285ECA9FDA98081EC
:1029100091812817390709F049C0A98EEA8EFB8EEC
:102920000C8F1D8FBE8FDF8EC8A2CE0149960E94EC
:10293000B5058BAB298D3A8D4B8D5C8D6D8D7E8D64
:10294000CE0101964C01ABA4BCA4CDA4DEA4EFA49F
:10295000F8A809A91AA98F8D98A10E949F03AA24FB
:10296000A394298D3A8D4B8D5C8D6D8D7E8D8F8DD1
:1029700098A12F3F354D41415E4763407105810568
:10298000910509F008F4A12CAF928BA8C980DA80D8
:10299000EB80FC800D811E812F81388549855A8509
:1029A0006B857C85C3010E9483100F90BFEF6B1A6B
:1029B0007B0AE9A5FAA53296FAA7E9A7F6E06F1611
:1029C000710409F07BCFF101EE0FFF1FE65CFA4FB7
:1029D000818592850E94110B80E0E5960FB6F894F0
:1029E000DEBF0FBECDBFDF91CF911F910F91FF9042
:1029F000EF90DF90CF90BF90AF909F908F907F909F
:102A00006F905F904F903F902F900895D10183E099
:102A1000AA0FBB1F8A95E1F7A65CBA4FFD01799614
:102A20005996DC9241825282A382E482F582068327
:102A3000178361E0872D962D0E94D60CCE018196DA
:102A40000E94B50589A72101440C551CF201E65CE2
:102A5000FA4F0184F285E02D29A13AA14BA15CA196
:102A60006DA17EA18FA1EF2B91F5A0909305B09061
:102A70009405C0909505D0909605E0909705F0904C
:102A800098050091990510919A05DE011D964D015A
:102A900098A50E949F031F9289A4A12CCD84DE8457
:102AA000EF84F88809891A892B893C894D895E89C8
:102AB0006F89788D872D962D0E948310F201E65C38
:102AC000FA4F818592850E94110B0F9085CFA090BF
:102AD0009B05B0909C05C0909D05D0909E05E09010
:102AE0009F05F090A0050091A1051091A205FE019F
:102AF0003D964F01CDCF81E070CFEF92FF920F93C3
:102B00001F93CF93DF93EC017B018A018881998128
:102B1000009729F02A813B812417350788F4B801F2
:102B20006F5F7F4F0E943030009791F099838883C8
:102B30001B830A832C813D81232B11F4FC0110821D
:102B40001D830C83B701888199810E94FF300CC0DE
:102B500088819981009711F00E94A72F198218820D
:102B60001D821C821B821A82CE01DF91CF911F91A0
:102B70000F91FF90EF900895FB0101900020E9F77D
:102B80003197AF01461B570B0C947D150F931F9384
:102B9000CF93DF93CDB7DEB762970FB6F894DEBF61
:102BA0000FBECDBF8C01CB01F801118210821382C0
:102BB0001282158214824AE0BE016F5F7F4F0E942D
:102BC0007F2ABE016F5F7F4FC8010E94BC156296CD
:102BD0000FB6F894DEBF0FBECDBFDF91CF911F912E
:102BE0000F910895FC0111821082138212821582C6
:102BF0001482FB0101900020E9F73197AF01461BD9
:102C0000570B0C947D1585ED8093BC0080913F049B
:102C100090914004A0914104B09142040796A11DF7
:102C2000B11D23E0B695A795979587952A95D1F77D
:102C30002091BC0024FD03C010923D0408954091F2
:102C40003F04509140046091410470914204452B2F
:102C5000462B472B69F30097A105B10541F025E309
:102C60002A95F1F700000197A109B109E1CF809100
:102C70003E040C9466091F920F920FB60F92112416
:102C80002F933F934F935F936F937F938F939F9374
:102C9000AF93BF93EF93FF9387E694E00E947F0783
:102CA000FF91EF91BF91AF919F918F917F916F9124
:102CB0005F914F913F912F910F900FBE0F901F90FA
:102CC00018951F920F920FB60F9211242F938F9386
:102CD0009F93EF93FF93E0917704F09178048081C4
:102CE000E0917D04F0917E0482FD1BC09081809173
:102CF00080048F5F8F7320918104821741F0E091EF
:102D00008004F0E0E959FB4F958F80938004FF9198
:102D1000EF919F918F912F910F900FBE0F901F9069
:102D200018958081F4CF1F920F920FB60F92112445
:102D30002F933F938F939F93AF93BF9380911005F1
:102D400090911105A0911205B09113053091E40303
:102D500023E0230F2D3758F50196A11DB11D2093B7
:102D6000E4038093100590931105A0931205B0938E
:102D700013058091E5039091E603A091E703B091DC
:102D8000E8030196A11DB11D8093E5039093E6032E
:102D9000A093E703B093E803BF91AF919F918F9108
:102DA0003F912F910F900FBE0F901F90189526E81E
:102DB000230F0296A11DB11DD2CF1F920F920FB605
:102DC0000F9211242F933F934F935F936F937F93B1
:102DD0008F939F93AF93BF93EF93FF938091B9002D
:102DE000887F803609F44AC0F0F5883209F4A7C01C
:102DF00018F5803109F49BC0B8F4882309F4F9C0B0
:102E0000883009F494C0FF91EF91BF91AF919F91E9
:102E10008F917F916F915F914F913F912F910F9083
:102E20000FBE0F901F901895883109F488C080322A
:102E300051F780933B0414C0803409F49DC040F4E2
:102E40008033B9F38833F9F680933B0485ECB0C046
:102E5000803509F485C0883509F496C0883499F620
:102E60000E940316D0CF883909F48CC038F5883712
:102E700029F050F4883611F0803729F683E08093EA
:102E80003D041092E30357C0883809F47BC08039B1
:102E900019F0803809F0B7CF8091E303803208F051
:102EA00071C0E091E30381E08E0F8093E303809192
:102EB000BB00F0E0ED53FC4F80833DC0803B39F018
:102EC000E0F4803A09F479C0883A09F09CCF84E0B4
:102ED00080933D041092C2031092C103E091E90374
:102EE000F091EA0309958091C10381110FC081E03F
:102EF0008093C1031092A10309C0803C09F4A6CFBE
:102F0000883C09F4A3CF883B09F07DCFE091C20350
:102F100081E08E0F8093C203F0E0EF55FC4F80817B
:102F20008093BB009091C2038091C10329C080911E
:102F300018048093BB0085EC8093BC0064CF909113
:102F40003A0480913904981758F5E0913A0481E0E9
:102F50008E0F80933A04F0E0E75EFB4F8081E9CF6B
:102F6000E0913A0481E08E0F80933A048091BB0097
:102F7000F0E0E75EFB4F808390913A048091390442
:102F80009817C8F285E8D8CFE0913A0481E08E0F17
:102F900080933A048091BB00F0E0E75EFB4F8083B2
:102FA00080913C0481115CCF81E08093170484EA16
:102FB0008093BC0010923D0426CF85EC8093BC002A
:102FC00010923D048091E303803230F4E091E303FA
:102FD000F0E0ED53FC4F10826091E30370E0E0916C
:102FE000EB03F091EC0383EC93E009951092E3037B
:102FF0000ACF10923B0434CF1F920F920FB60F925C
:1030000011242F933F934F935F936F937F938F93ED
:103010009F93AF93BF93CF93DF93EF93FF938091F1
:1030200039050E943708EC01809138050E94370865
:10303000909137059F70CC0FDD1FC82B24E0929F25
:10304000C0011124815B9E4FC80FD92FD11D8881EB
:103050008093370580738031B9F481E090E00E945D
:10306000480EFF91EF91DF91CF91BF91AF919F916A
:103070008F917F916F915F914F913F912F910F9021
:103080000FBE0F901F901895803259F78FEF9FEF6A
:10309000E6CF10926A041092690488EE93E0A0E0F3
:1030A000B0E080936B0490936C04A0936D04B09394
:1030B0006E042FE631E0309368042093670425EC1A
:1030C00030E0309374042093730424EC30E03093A8
:1030D00076042093750420EC30E03093780420933C
:1030E000770421EC30E030937A042093790422ECC9
:1030F00030E030937C0420937B0426EC30E0309366
:103100007E0420937D04109280041092810410921A
:103110008204109283041092070510920605809392
:10312000080590930905A0930A05B0930B0581E863
:1031300091E090930505809304051092AF051092DD
:10314000AE0589E991E09093AD058093AC0584E0EC
:103150008093B0058FEF8093B10586E08093B20530
:1031600087E08093B30588E08093B40589E080937D
:10317000B5058AE08093B6051092B7051092B805A0
:103180001092B9051092BA0561E084E00E948E08A1
:103190008091B1058F3F19F061E00E948E0861E0D7
:1031A0008091B2050E948E081092BB0581E00E94BA
:1031B000CF0D80E68093AB0510923A0510923B0547
:1031C00010923C0510923D0510923E0510923F056D
:1031D00010924005109241051092420580E498E754
:1031E000ADE7B1E08093A3059093A405A093A50556
:1031F000B093A60583E08093380582E0809339057B
:1032000060E083E00E948E0860E0809139050E94B2
:103210008E0861E0809138050E94600861E080912D
:1032200039050E9460081092370564E572E081E379
:1032300095E00E94F2156CE572E08BE295E00E9449
:10324000F2152FB7F8948091100590911105A09177
:103250001205B09113052FBF90932305809322058B
:103260001092250510922405109226058FE891E012
:10327000909321058093200580E190E090932805AC
:103280008093270510922A051092290562E00E947A
:103290008E0864E572E08AE195E00E94F21564E52B
:1032A00072E084E195E00C94F215CF93DF9300D0A7
:1032B00000D000D0CDB7DEB7789484B5826084BDED
:1032C00084B5816084BD85B5826085BD85B581602A
:1032D00085BD80916E00816080936E0010928100A8
:1032E0008091810082608093810080918100816063
:1032F0008093810080918000816080938000809124
:10330000B10084608093B1008091B00081608093AF
:10331000B00080917A00846080937A0080917A0076
:10332000826080937A0080917A00816080937A0035
:1033300080917A00806880937A001092C100E091B9
:103340007704F091780482E08083E0917304F09137
:1033500074041082E0917504F091760487E680830E
:1033600010927F04E0917B04F0917C0486E08083DE
:10337000E0917904F0917A04808180618083E0910A
:103380007904F0917A04808188608083E0917904E7
:10339000F0917A04808180688083E0917904F091D3
:1033A0007A0480818F7D808382E00E94CF0D0E940D
:1033B000C70D1092F6031092F50310924404109278
:1033C00066040E94480985EF96E09093EA03809393
:1033D000E90386EF96E09093EC038093EB0362E0C1
:1033E0008FE00E948E0862E080E10E948E0861E01A
:1033F00085E00E948E0860E084E10E948E0868E209
:1034000071E080E00E94160F60E271E081E00E94AE
:10341000160F68E171E082E00E94160F60E171E032
:1034200083E00E94160F90E080E00E94D82B60930A
:103430000C0170930D0180930E0190930F01672B87
:10344000682B692B61F480E498E7ADE7B1E08093E5
:103450000C0190930D01A0930E01B0930F0184E035
:1034600090E00E94D82B60934001709341018093BB
:10347000420190934301672B682B692B61F480E82C
:1034800096E9A8E9B0E08093400190934101A093B0
:103490004201B093430188E090E00E94D82B6093F2
:1034A00038017093390180933A0190933B01672B67
:1034B000682B692B61F480E896E9A8E9B0E0809375
:1034C000380190933901A0933A01B0933B0161E038
:1034D00080E00E94B80D84EA91E00E94A20F609102
:1034E0000C0170910D0180910E0190910F014AE045
:1034F0000E94540F68EB7BE080E090E00E94EF08B0
:103500000E94C70D61E081E00E94B80D8BEA91E056
:103510000E94A20F609138017091390180913A01A7
:1035200090913B014AE00E94540F68EB7BE080E001
:1035300090E00E94EF0861E080E00E94B80D0E94D8
:10354000C70D81EB91E00E94A20F60914001709144
:10355000410180914201909143014AE00E94540F41
:1035600068EB7BE080E090E00E94EF080E94C70DCE
:103570008CE090E00E94D82B60933201709333016D
:103580008093340190933501C0900C01D0900D01CF
:10359000E0900E01F0900F011092F6031092F503E7
:1035A00010924404109266040E94480985EF96E048
:1035B0009093EA038093E90386EF96E09093EC03FF
:1035C0008093EB0362E987EB0E94F60AC114D104F1
:1035D000E104F104D1F08FE00E94AC0B682F6F730F
:1035E00001E8C01603ECD00609ECE00601E0F006A5
:1035F00008F0B6C1C092A305D092A405E092A5053B
:10360000F092A6058FE00E94F60A1092A70510928C
:10361000A8051092A9051092AA0560E880E10E9411
:10362000F60A60E881E10E94F60A60E882E10E9401
:10363000F60A60E883E10E94F60A60E884E10E94ED
:10364000F60A60E885E10E94F60A60E886E10E94D9
:10365000F60A60E887E10E94F60A6CE080E10E94C9
:10366000F60A6CE081E10E94F60A6CE082E10E94B9
:10367000F60A6CE083E10E94F60A6CE084E10E94A5
:10368000F60A6CE085E10E94F60A6CE086E10E9491
:10369000F60A6CE087E10E94F60A10E000E020E004
:1036A00030E24FE550EA62E170E080E090E00E9495
:1036B0006E1101E010E020E030E24FE550EA62E1F7
:1036C00070E080E090E00E946E111092440510922C
:1036D0004305109246051092450510924805109238
:1036E000470510924A051092490510924C05109218
:1036F0004B0510924E0510924D0581E090E090939D
:10370000500580934F05909352058093510570E0CA
:1037100060E090E080E00E94EE0C70E060E081E00C
:1037200090E00E94EE0C70E060E082E090E00E9489
:10373000EE0C70E060E083E090E00E94EE0C70E040
:1037400060E084E090E00E94EE0C70E060E085E0D4
:1037500090E00E94EE0C61E070E086E090E00E9454
:10376000EE0C61E070E087E090E00E94EE0C60E01B
:1037700082EA0E94F60A60E083EA0E94F60A60E0AC
:1037800084EA0E94F60A90E080E00E94110B60E853
:1037900081EB0E94F60A03E515E0F12CE12CD8013B
:1037A0001C9211961C92119712961C9212971396C6
:1037B0001C92139714961C92149715961C921597A9
:1037C00016961C92169717961C92085F1F4F60E082
:1037D000C7010E94D60CBFEFEB1AFB0AE8E0EE1619
:1037E000F104E9F610E000E020E030E24FE550EAB5
:1037F00062E170E080E090E00E946E1162E08BE098
:103800000E948E0880916800846080936800809197
:103810006D008C6080936D0078948BE00E94370877
:10382000892B09F0F5C48091320190913301A09168
:103830003401B09135018093080190930901A09360
:103840000A01B0930B010E94C70D60E080E00E9466
:10385000B80D87EB91E00E94A20F68EB7BE080E05F
:1038600090E00E94EF0861E080E00E94B80D80ECDB
:1038700091E00E94A20F50E4C52E58E7D52E5DE7D7
:10388000E52EFF24F39480913601909137011816AC
:1038900019060CF0F8C08FE00E943708892B09F058
:1038A000E7C060E080E00E94B80D8EEC91E00E94DD
:1038B000A20F61E080E00E94B80D8FED91E00E94C0
:1038C000A20F68E873E180E090E00E94EF080E9498
:1038D000C70D60E080E00E94B80D8FEE91E00E947D
:1038E000A20F61E080E00E94B80D80E092E00E94AB
:1038F000A20F68E873E180E090E00E94EF08C092B8
:103900003201D0923301E0923401F092350110E09F
:1039100000E020E039EF42E055E960E070E080E04F
:1039200090E00E9462130E94C70D61E080E00E9457
:10393000B80D8FEE91E00E94A20F0E94AF0F8FE0B2
:103940000E943708892B09F441C0809144018823E3
:1039500021F00E94AF0F109244010E944D0BEFCF57
:10396000D701C6018158934CA94CB1408038934C83
:10397000A94CB14070F4F694E794D794C794C092E0
:10398000A305D092A405E092A505F092A605606477
:1039900039CED701C60181509748A349B34081155C
:1039A0009A45A246B24008F02DCE72E0F694E79414
:1039B000D794C7947A95D1F7C092A305D092A40565
:1039C000E092A505F092A60560681CCE61E081E05A
:1039D0000E94B80D609132017091330180913401E1
:1039E000909135014AE00E94540F81E192E00E94DB
:1039F000A20F68EB7BE080E090E00E94EF0861E0BE
:103A000080E00E94B80D81E292E00E94A20F80E166
:103A10000E943708892B31F18FE00E943708892BEB
:103A2000B1F74091320150913301609134017091AE
:103A3000350190E080E00E94DE2B61E080E00E9492
:103A4000B80D82E392E00E94A20F60ED77E080E083
:103A500090E00E94EF0861E080E00E94B80D83E4EE
:103A600092E0D3CF0E94C70D109237011092360119
:103A700080E10E943708892B09F005CF10923701A9
:103A80001092360100CF0E94C70D81E090E0909324
:103A900037018093360160E080E00E94B80D85E533
:103AA00092E00E94A20F68EB7BE080E090E00E9431
:103AB000EF0861E080E00E94B80D80EC91E00E9488
:103AC000A20F38E3C32E32EAD32E38E9E32EF12CCD
:103AD00040EE842E4CEE942E44E0A42EBB24B394EE
:103AE0008091360190913701181619060CF0A6C185
:103AF0008FE00E943708892B09F095C110E000E0A3
:103B000020E837E84CEE55E660E070E080E090E0B9
:103B10000E946213609140017091410180914201C5
:103B20009091430124E630E040E050E00E94E92D0E
:103B300002E010E00E94621360E080E00E94B80D95
:103B400080E692E00E94A20F61E080E00E94B80D42
:103B500080E792E00E94A20F6091400170914101C4
:103B600080914201909143014AE00E94540F68E81D
:103B700073E180E090E00E94EF080E94C70D60E0D2
:103B800080E00E94B80D89E792E00E94A20F61E0F8
:103B900080E00E94B80D88E892E00E94A20F68E8D9
:103BA00073E180E090E00E94EF08C0923201D09271
:103BB0003301E0923401F09235010E94C70D61E0BB
:103BC00080E00E94B80D8FEE91E00E94A20F0E944B
:103BD000AF0F8FE00E943708892BE9F080914401F4
:103BE000882321F00E94AF0F109244010E944D0BD8
:103BF00060913201709133018091340190913501CF
:103C000024E630E040E050E00E94E92D02E010E0C0
:103C10000E946213DECF8091320190913301A09116
:103C20003401B09135018093400190934101A093FC
:103C30004201B09343010E94C70D60E080E00E9402
:103C4000B80D87E992E00E94A20F61E080E00E9437
:103C5000B80D88EA92E00E94A20F68E873E180E064
:103C600090E00E94EF0861E080E00E94B80D8FEEC6
:103C700091E00E94A20F0E94C70D809232019092A3
:103C80003301A0923401B09235010E94AF0F61E080
:103C900080E00E94B80D8FEE91E00E94A20F8FE0AD
:103CA0000E943708892BE9F080914401882321F094
:103CB0000E94AF0F109244010E944D0B609132019F
:103CC00070913301809134019091350124E630E008
:103CD00040E050E00E94E92D10E000E00E946213F5
:103CE000DECF60E080E00E94B80D89EB92E00E9498
:103CF000A20F61E080E00E94B80D8AEC92E00E9481
:103D0000A20F68E873E180E090E00E94EF080E9453
:103D1000C70D8091400190914101A0914201B09165
:103D200043018093320190933301A0933401B09307
:103D300035010E94AF0F61E080E00E94B80D8FEE68
:103D400091E00E94A20F8FE00E943708892BE9F0D2
:103D500080914401882321F00E94AF0F109244010A
:103D60000E944D0B609132017091330180913401BA
:103D70009091350124E630E040E050E00E94E92DCA
:103D800002E010E00E946213DECF61E081E00E9459
:103D9000B80D60913201709133018091340190919E
:103DA00035014AE00E94540F8BED92E00E94A20F71
:103DB00068EB7BE080E090E00E94EF0861E080E04B
:103DC0000E94B80D83EE92E00E94A20F80E10E9453
:103DD0003708892B31F18FE00E943708892BB1F722
:103DE000409132015091330160913401709135015D
:103DF00084E090E00E94DE2B61E080E00E94B80D3C
:103E000085EF92E00E94A20F60ED77E080E090E005
:103E10000E94EF0861E080E00E94B80D83E492E028
:103E2000D3CF0E94C70D80E10E943708892B09F08B
:103E300057CE109237011092360152CE0E94C70D14
:103E400081E090E0909337018093360160E080E05C
:103E50000E94B80D84E093E00E94A20F68EB7BE023
:103E600080E090E00E94EF0861E080E00E94B80DE1
:103E700080EC91E00E94A20F98EFC92E92E8D92E13
:103E800098E9E92EF12C20E2822E20E4922E2CE2F9
:103E9000A22EB12C80913601909137011816190687
:103EA0000CF09EC18FE00E943708892B09F08DC16C
:103EB00010E000E020E83CE049E451E160E070E01F
:103EC00080E090E00E9462136091380170913901A6
:103ED00080913A0190913B0124E630E040E050E0CF
:103EE0000E94E92D02E010E00E94621360E080E091
:103EF0000E94B80D8FE093E00E94A20F61E080E085
:103F00000E94B80D81E792E00E94A20F60913801F3
:103F10007091390180913A0190913B014AE00E94F1
:103F2000540F68E873E180E090E00E94EF080E947F
:103F3000C70D60E080E00E94B80D89E792E00E9422
:103F4000A20F61E080E00E94B80D88E892E00E9434
:103F5000A20F68E873E180E090E00E94EF08C09251
:103F60003201D0923301E0923401F09235010E9487
:103F7000C70D61E080E00E94B80D8FEE91E00E94D5
:103F8000A20F0E94AF0F8FE00E943708892BE9F043
:103F900080914401882321F00E94AF0F10924401C8
:103FA0000E944D0B60913201709133018091340178
:103FB0009091350124E630E040E050E00E94E92D88
:103FC00002E010E00E946213DECF809132019091F6
:103FD0003301A0913401B091350180933801909361
:103FE0003901A0933A01B0933B010E94C70D60E0F4
:103FF00080E00E94B80D8EE193E00E94A20F61E084
:1040000080E00E94B80D8EE293E00E94A20F68E863
:1040100073E180E090E00E94EF080E94C70D61E02C
:1040200080E00E94B80D8DE393E00E94A20F809281
:10403000320190923301A0923401B09235010E9476
:10404000AF0F8FE00E943708892BE9F0809144017F
:10405000882321F00E94AF0F109244010E944D0B63
:10406000609132017091330180913401909135015A
:1040700024E630E040E050E00E94E92D10E000E04E
:104080000E946213DECF60E080E00E94B80D89EBF1
:1040900092E00E94A20F61E080E00E94B80D8AECDD
:1040A00092E00E94A20F68E873E180E090E00E9435
:1040B000EF080E94C70D8091380190913901A091BD
:1040C0003A01B0913B018093320190933301A09368
:1040D0003401B09335010E94AF0F61E080E00E948F
:1040E000B80D8FEE91E00E94A20F8FE00E9437087A
:1040F000892BE9F080914401882321F00E94AF0FC1
:10410000109244010E944D0B609132017091330175
:10411000809134019091350124E630E040E050E098
:104120000E94E92D02E010E00E946213DECF61E000
:1041300081E00E94B80D609132017091330180914D
:104140003401909135014AE00E94540F8BED92E0CA
:104150000E94A20F68EB7BE080E090E00E94EF08F5
:1041600061E080E00E94B80D8EE493E00E94A20F0F
:1041700080E10E943708892B31F18FE00E943708D7
:10418000892BB1F740913201509133016091340194
:104190007091350188E090E00E94DE2B61E080E0C4
:1041A0000E94B80D85EF92E00E94A20F60ED77E0CB
:1041B00080E090E00E94EF0861E080E00E94B80D8E
:1041C00083E492E0D3CF0E94C70D80E10E943708BC
:1041D000892B09F05FCE10923701109236015ACE2A
:1041E0008091080190910901A0910A01B0910B0101
:1041F0008093320190933301A0933401B093350141
:104200000E94C70D81E090E09093370180933601C2
:104210008091400190914101A0914201B0914301F0
:1042200080933C0190933D01A0933E01B0933F01E8
:104230000E94C70D0E94AF0F80E2882E8FE2982E59
:1042400084E1A82EBB24B3942FB7F8948091100575
:1042500090911105A0911205B09113052FBF4091C7
:10426000F1035091F2036091F3037091F4038C0118
:104270009D01041B150B260B370BB901A801443F08
:1042800051406105710510F40C94342A8093F103B8
:104290009093F203A093F303B093F40386E4809326
:1042A0007C0080917A00806480937A0080917A000B
:1042B00086FDFCCF8091780060917900762F682F81
:1042C000072E000C880B990B0E94BB2A20E030E4DB
:1042D0004CE955E40E941A2B20E030E040E85AE314
:1042E0000E941A2B60934501709346018093470109
:1042F0009093480120E030E040E850E40E94B42A66
:1043000087FF0EC061E070E0CE0101960E94C615E5
:10431000CE0101960E943E10CE0101960E947B10B4
:10432000C0904501D0904601E0904701F0904801CF
:1043300020E030E040E850E4C701B6010E94642D5F
:1043400087FD18C020E030E040E051E4C701B6012D
:104350000E94B42A87FF0EC061E070E0CE01019692
:104360000E94C615CE0101960E943E10CE01019614
:104370000E947B10C0904501D0904601E09047011B
:10438000F090480120E030E040E051E4C701B60180
:104390000E94642D87FD18C020E030E040E451E425
:1043A000C701B6010E94B42A87FF0EC062E070E028
:1043B000CE0101960E94C615CE0101960E943E10C4
:1043C000CE0101960E947B10C0904501D09046011D
:1043D000E0904701F090480120E030E040E451E4F3
:1043E000C701B6010E94642D87FD18C020E030E0AF
:1043F00040EA51E4C701B6010E94B42A87FF0EC00B
:1044000063E070E0CE0101960E94C615CE010196D0
:104410000E943E10CE0101960E947B10C090450183
:10442000D0904601E0904701F090480120E030E054
:1044300040EA51E4C701B6010E94642D87FD18C00F
:1044400020E030E04CE152E4C701B6010E94B42AFA
:1044500087FF0EC064E070E0CE0101960E94C61591
:10446000CE0101960E943E10CE0101960E947B1063
:10447000C0904501D0904601E0904701F09048017E
:1044800020E030E04CE152E4C701B6010E94642D07
:1044900087FD18C020E030E044E952E4C701B601CE
:1044A0000E94B42A87FF0EC065E070E0CE0101963D
:1044B0000E94C615CE0101960E943E10CE010196C3
:1044C0000E947B10C0904501D0904601E0904701CA
:1044D000F090480120E030E044E952E4C701B60121
:1044E0000E94642D87FD10C020E030E044E153E4D9
:1044F000C701B6010E94B42A87FF06C060E673E0D8
:104500008AE195E00E94BC1520E030E044E153E4EC
:10451000C701B6010E94642D87FD10C020E030E085
:1045200046E953E4C701B6010E94B42A87FF06C0DA
:1045300064E673E08AE195E00E94BC1520E030E07B
:1045400046E953E4C701B6010E94642D87FD10C0FF
:1045500020E030E445E154E4C701B6010E94B42AEA
:1045600087FF06C068E673E08AE195E00E94BC150B
:1045700020E030E445E154E4C701B6010E94642D17
:1045800087FD10C020E030EC44E954E4C701B601D7
:104590000E94B42A87FF06C06CE673E08AE195E0CA
:1045A0000E94BC1520E030EC44E954E4C701B60198
:1045B0000E94642D87FD10C020E030E04BE655E4FA
:1045C000C701B6010E94B42A87FF06C060E773E006
:1045D0008AE195E00E94BC1520E030E04BE655E40E
:1045E000C701B6010E94642D87FD06C064E773E031
:1045F0008AE195E00E94BC158091180590911905FB
:10460000C0901E05D0901F05E0901A05F0901B0584
:104610008C159D0509F079C68091140590911505BA
:10462000009709F464C6E114F10441F4C114D10403
:1046300009F485C6FC01808190E065C6B7010E943F
:10464000F63061C68091140590911505009711F020
:104650000E94A72F109215051092140510921905AB
:1046600010921805109217051092160558C6821759
:10467000930709F412C180912605882389F180915E
:10468000240590912505059759F58091EF039091A8
:10469000F00301969093F0038093EF0321E02093C1
:1046A0004401059731F481E090E09093F00380930A
:1046B000EF038091EF039091F0038230910509F4AC
:1046C00010C10CF0F9C06CE572E0019709F40EC15D
:1046D00061E080E00E94B80D8BE295E00E94250722
:1046E00080912605882309F42AC28091240590919F
:1046F0002505079709F023C28091ED039091EE0301
:1047000001968A30910509F406C19093EE038093D7
:10471000ED03E090ED03F090EE0311E0E116F104FB
:1047200009F0FCC080E295E7A8E3B0E08093320195
:1047300090933301A0933401B093350188E793E05F
:104740000E943B0F882361F080E19DEDA5E3B0E07E
:104750008093320190933301A0933401B0933501DB
:104760008CE793E00E943B0F882361F088E095E896
:10477000A6E3B0E08093320190933301A09334011B
:10478000B093350196E0E916F10409F018C100E88C
:104790001CE723E431E000933201109333012093AE
:1047A00034013093350188E793E00E943B0F882362
:1047B00061F060E774EE80E491E060933201709301
:1047C000330180933401909335018CE793E00E948C
:1047D0003B0F882309F4A8C180E590E9A1E4B1E08A
:1047E0008093320190933301A0933401B09335014B
:1047F0009BC18217930709F053C0E0912005F09107
:10480000210580819181081719070CF434CF82E0CB
:1048100090E037C08217930709F045C0E09120056A
:10482000F091210584819581081719070CF423CF95
:1048300088E090E026C082179307C1F1E09120053F
:10484000F091210582819381081719070CF413CF89
:1048500085E090E016C08217930759F5E091200596
:10486000F091210580819181081719070CF403CF7D
:1048700087E090E006C08217930709F4FCCE89E038
:1048800090E0D0922305C092220590932505809355
:10489000240581E080932605EECE81E090E0F1CF03
:1048A00090E080E0EECF83E090E0EBCF86E090E018
:1048B000E8CF84E090E0E5CF83309105A9F06CE784
:1048C00073E0049709F004CF8BE295E00E94BC15D9
:1048D0008091380190913901A0913A01B0913B014A
:1048E00011C06BE073E0F0CF68E773E08BE295E016
:1048F0000E94BC158091400190914101A09142011C
:10490000B091430180933C0190933D01A0933E01FF
:10491000B0933F01DDCE81E090E0F7CE22E0E216D9
:10492000F10451F580E696E5ACE6B0E08093320103
:1049300090933301A0933401B093350188E793E05D
:104940000E943B0F882361F080EF94E4ABE6B0E077
:104950008093320190933301A0933401B0933501D9
:104960008CE793E00E943B0F882309F40BCF80ED86
:1049700090EFABE6B0E0FECE33E0E316F10409F0D1
:104980004DC080E29DE1AAE9B0E0809332019093AE
:104990003301A0933401B09335018CE793E00E947A
:1049A0003B0F882361F080EC99EAAAE9B0E080939C
:1049B000320190933301A0933401B093350197E015
:1049C000E916F10409F05FC000E01BE62AE731E0D8
:1049D0000093320110933301209334013093350159
:1049E00088E793E00E943B0F882361F060E370EE5C
:1049F0008AE791E060933201709333018093340130
:104A0000909335018CE793E00E943B0F882309F4D3
:104A10008BC080EF97E3ACE7B1E0E2CE64E0E6164E
:104A2000F10409F054C080EC9CEAA8EDB0E080935A
:104A3000320190933301A0933401B093350188E79C
:104A400093E00E943B0F882361F080EB94E1A6ED98
:104A5000B0E08093320190933301A0933401B0937E
:104A600035018CE793E00E943B0F882361F080E9D9
:104A700090ECA6EDB0E08093320190933301A093C7
:104A80003401B093350198E0E916F10409F085C3CB
:104A900000EE1DE923EA31E0009332011093330167
:104AA00020933401309335018CE793E00E943B0F53
:104AB0008823D1F168EE77E080EA91E060933201DB
:104AC0007093330180933401909335012DC075E0CC
:104AD000E716F10409F056CE80923201909233012C
:104AE000A0923401B092350188E793E00E943B0F19
:104AF000882361F080EB9DE1A3E1B1E08093320176
:104B000090933301A0933401B09335018CE793E087
:104B10000E943B0F882341F0809232019092330132
:104B2000A0923401B092350161E080E00E94B80D9E
:104B30008BE295E00E94250781E0809344018091FB
:104B40002605882309F44AC0809124059091250503
:104B5000089709F043C00E94C70D60E080E00E9402
:104B6000B80D80E893E00E94A20F68EB7BE080E044
:104B700090E00E94EF0861E080E00E94B80D81E9BA
:104B800093E00E94A20F8091360190913701181690
:104B9000190604F58FE00E943708892B09F02CC311
:104BA000409132015091330160913401709135018F
:104BB0008CE090E00E94DE2B61E080E00E94B80D66
:104BC00085EF92E00E94A20F60ED77E080E090E038
:104BD0000E94EF080E94C70D0E94AF0F8091440110
:104BE000882309F4C9C288E793E00E943B0F882319
:104BF00081F08091400190914101A0914201B091DA
:104C0000430180933C0190933D01A0933E01B093FA
:104C10003F018BE093E00E943B0F882381F080915D
:104C2000380190913901A0913A01B0913B018093F4
:104C30003C0190933D01A0933E01B0933F018CE570
:104C400092E00E943B0F882381F080914001909177
:104C50004101A0914201B091430180933C019093A6
:104C60003D01A0933E01B0933F018CE793E00E9489
:104C70003B0F882381F08091380190913901A091F8
:104C80003A01B0913B0180933C0190933D01A09388
:104C90003E01B0933F0160913201709133018091E8
:104CA0003401909135010E94B92A20E034E244E7B2
:104CB00059E40E94BC2C6B017C0120E030E040ED07
:104CC00050E40E94B42A87FF06C081E090E09093F0
:104CD00031018093300120E030E040ED50E4C70125
:104CE000B6010E94642D87FD2FC02AE939E949E207
:104CF00051E4C701B6010E94B42A87FF25C021EE06
:104D00003AE744E851E4C701B6010E941A2B20E0BB
:104D100030E047ED52E40E944F2C2B013C0120E093
:104D200030E0A9010E94642D20E030E040E05FE324
:104D300087FD69C2C301B2010E94502C0E942E2D32
:104D400070933101609330012AE939E949E251E475
:104D5000C701B6010E94642D87FD2FC020E030E01E
:104D600040E551E4C701B6010E94B42A87FF25C07F
:104D70002FE832EC45E351E4C701B6010E941A2B3B
:104D800029E23CE541E552E40E944F2C2B013C0115
:104D900020E030E0A9010E94642D20E030E040E0F6
:104DA0005FE387FD35C2C301B2010E94502C0E940F
:104DB0002E2D709331016093300120E030E040E50A
:104DC00051E4C701B6010E94642D87FD2FC020E089
:104DD00030E040E651E4C701B6010E94B42A87FFE3
:104DE00025C025E83BEE41EC50E4C701B6010E9426
:104DF0001A2B2DE33AE047E851E40E94502C2B0196
:104E00003C0120E030E0A9010E94642D20E030E068
:104E100040E05FE387FD01C2C301B2010E94502C54
:104E20000E942E2D709331016093300120E030E01C
:104E300040E651E4C701B6010E94642D87FD2FC0F2
:104E400020E030E040EA51E4C701B6010E94B42AF4
:104E500087FF25C027E139ED4EE051E4C701B601D7
:104E60000E941A2B20E030E048EB51E40E944F2CC6
:104E70002B013C0120E030E0A9010E94642D20E0DC
:104E800030E040E05FE387FDCDC1C301B2010E9485
:104E9000502C0E942E2D709331016093300120E040
:104EA00030E040EA51E4C701B6010E94642D87FD5D
:104EB0002FC020E030E048EB51E4C701B6010E946A
:104EC000B42A87FF25C028EF33E545E051E4C70148
:104ED000B6010E941A2B2CE53FE84AE251E40E94F9
:104EE0004F2C2B013C0120E030E0A9010E94642DF1
:104EF00020E030E040E05FE387FD99C1C301B201EB
:104F00000E94502C0E942E2D70933101609330012D
:104F100020E030E048EB51E4C701B6010E94642D67
:104F200087FD2FC020E030E040ED51E4C701B6011D
:104F30000E94B42A87FF25C02FE335E34AEA50E4F4
:104F4000C701B6010E941A2B27ED33EA4AE652E464
:104F50000E94502C2B013C0120E030E0A9010E946E
:104F6000642D20E030E040E05FE387FD65C1C301D0
:104F7000B2010E94502C0E942E2D7093310160933B
:104F8000300120E030E040ED51E4C701B6010E945D
:104F9000642D87FD2FC020E030E048EE51E4C701CA
:104FA000B6010E94B42A87FF25C028E631E949EE00
:104FB00050E4C701B6010E941A2B2AE534E643EEFD
:104FC00050E40E94502C2B013C0120E030E0A9016C
:104FD0000E94642D20E030E040E05FE387FD31C1B6
:104FE000C301B2010E94502C0E942E2D70933101FA
:104FF0006093300120E030E048EE51E4C701B60193
:105000000E94642D87FD2FC020E030E048EF51E47E
:10501000C701B6010E94B42A87FF25C026EF38E2F7
:105020004CE351E4C701B6010E941A2B2AE939E981
:1050300043EF52E40E944F2C2B013C0120E030E072
:10504000A9010E94642D20E030E040E05FE387FD8D
:10505000FDC0C301B2010E94502C0E942E2D7093FE
:1050600031016093300120E030E048EF51E4C701A6
:10507000B6010E94642D87FD2FC020E030E04CEF88
:1050800051E4C701B6010E94B42A87FF25C024EA73
:1050900030E741E951E4C701B6010E941A2B26E628
:1050A00036E640EA53E40E944F2C2B013C0120E0FD
:1050B00030E0A9010E94642D20E030E040E05FE391
:1050C00087FDC9C0C301B2010E94502C0E942E2D41
:1050D000709331016093300120E030E04CEF51E4F7
:1050E000C701B6010E94642D87FD06C08FEF90E0D6
:1050F000909331018093300161E082E00E94B80D0D
:10510000009130011091310161E085E00E948E082C
:105110000115110509F0A4C060E085E00E94600857
:105120000E94AF0FC0903C01D0903D01E0903E0145
:10513000F0903F0160913201709133018091340110
:10514000909135016C0D7D1D8E1D9F1D24E630E074
:1051500040E050E00E94E92D10E000E00E94621360
:10516000C701B60124E630E040E050E00E94E92D9E
:1051700002E010E00E946213109244010E944D0B65
:1051800080E090E0892B09F45FC80E946B078823B8
:1051900009F452C80E9400004FC879E0E716F104F4
:1051A00009F0C2CC80E290EEA2EBB1E08093320134
:1051B00090933301A0933401B093350188E793E0D5
:1051C0000E943B0F882361F000E314EB2BEA31E0EF
:1051D0000093320110933301209334013093350151
:1051E0008CE793E00E943B0F882309F49DCC60E19B
:1051F00070E68CEA91E062CC80E10E943708892B4E
:1052000009F0C1CCE7CCC301B2010E944F2C96CD6E
:10521000C301B2010E944F2CCACDC301B2010E944A
:105220004F2CFECDC301B2010E944F2C32CEC301E0
:10523000B2010E944F2C66CEC301B2010E944F2CD6
:105240009ACEC301B2010E944F2CCECEC301B2014F
:105250000E944F2C02CFC301B2010E944F2C36CFC7
:105260000F3F110511F461E058CFE3EBF0E0E4915A
:10527000E33019F140F4E130B1F0E230C9F0003828
:1052800011058CF749CFE73011F1E83041F1E430F6
:10529000B1F78091800080628093800010938B0032
:1052A00000938A003DCF84B5806884BD07BD38CFA8
:1052B00084B5806284BD08BD33CF80918000806852
:1052C00080938000109389000093880029CF8091FB
:1052D000B00080688093B0000093B30021CF80912C
:1052E000B00080628093B0000093B40019CFE11445
:1052F000F10429F1C114D10411F1D7018C9190E08E
:10530000919581959109892BD1F0E114F10409F46B
:1053100099C9A601B70184E195E00E947D1561E07D
:1053200085E00E94B80D89E492E00E94A20F61E03E
:1053300085E00E94B80D8AE195E00E942507C090A3
:105340004501D0904601E0904701F090480120E0EF
:1053500030E048EA51E4C701B6010E94642D87FDA0
:1053600009C061E089E00E94B80D63E08CEA95E035
:105370000E94100F20E030E040E352E4C701B60184
:105380000E94642D87FD09C061E08AE00E94B80D8B
:1053900063E08CEA95E00E94100F20E030E046EADE
:1053A00052E4C701B6010E94642D87FD09C061E087
:1053B0008BE00E94B80D62E08CEA95E00E94100F2D
:1053C00020E030E047E253E4C701B6010E94642DBB
:1053D00087FD09C061E08CE00E94B80D61E08CEAB5
:1053E00095E00E94100F20E030E049EA53E4C70145
:1053F000B6010E94642D87FD09C061E08DE00E9426
:10540000B80D61E08CEA95E00E94100F20E030E0DA
:1054100048E254E4C701B6010E94642D87FD09C02B
:1054200061E08EE00E94B80D60E08CEA95E00E9499
:10543000100F20E030E847EA54E4C701B6010E94AB
:10544000642D87FD09C061E08FE00E94B80D60E027
:105450008CEA95E00E94100F8091BC058D7F8093AF
:10546000BC0588600E94B20D809127050E94370814
:105470002091290530912A0510922605821793075D
:1054800039F04091240550912505452B09F4F3C8C6
:105490004FB7F894C0901005D0901105E090120518
:1054A000F09013054FBF40912205509123058601CE
:1054B000041B150BE0912405F0912505E930F10559
:1054C00008F0EEC9EA59F54D0C948B2D3723F923DA
:1054D0000A2459241B2450242B243B243B2484E1FC
:1054E00095E00E947B108AE195E00E947B108BE2A0
:1054F00095E00E947B1081E395E00C947B10BB2724
:105500004A3031F4992322F4BDE2909581959F4F62
:105510000C948B2ABB27FB015527AA27880F991FBC
:10552000AA1FA41710F0A41B83955051B9F7A05DD2
:10553000AA3308F0A95DA193009779F7B111B1934F
:105540001192CB010C94A42ADC01FC01672F71910C
:105550007723E1F7329704C07C916D937083629159
:10556000AE17BF07C8F308950E94F62A08F481E039
:105570000895E89409C097FB3EF490958095709546
:1055800061957F4F8F4F9F4F9923A9F0F92F96E98F
:10559000BB279395F695879577956795B795F11104
:1055A000F8CFFAF4BB0F11F460FF1BC06F5F7F4FA1
:1055B0008F4F9F4F16C0882311F096E911C07723B3
:1055C00021F09EE8872F762F05C0662371F096E8BC
:1055D000862F70E060E02AF09A95660F771F881F8B
:1055E000DAF7880F9695879597F90895990F00082F
:1055F000550FAA0BE0E8FEEF16161706E807F907A5
:10560000C0F012161306E407F50798F0621B730B3F
:10561000840B950B39F40A2661F0232B242B252BC0
:1056200021F408950A2609F4A140A6958FEF811D63
:10563000811D08950E942D2B0C949E2B0E94902B6F
:1056400038F00E94972B20F0952311F00C94872BB3
:105650000C948D2B11240C94D22B0E94AF2B70F341
:10566000959FC1F3950F50E0551F629FF001729F07
:10567000BB27F00DB11D639FAA27F00DB11DAA1F16
:10568000649F6627B00DA11D661F829F2227B00D63
:10569000A11D621F739FB00DA11D621F839FA00DEE
:1056A000611D221F749F3327A00D611D231F849F3E
:1056B000600D211D822F762F6A2F11249F57504095
:1056C0009AF0F1F088234AF0EE0FFF1FBB1F661F10
:1056D000771F881F91505040A9F79E3F510580F0D9
:1056E0000C94872B0C94D22B5F3FE4F3983ED4F3B9
:1056F000869577956795B795F795E7959F5FC1F77D
:10570000FE2B880F911D9695879597F9089597F927
:105710009F6780E870E060E008959FEF80EC089557
:1057200000240A9416161706180609060895002480
:105730000A9412161306140605060895092E0394FA
:10574000000C11F4882352F0BB0F40F4BF2B11F46E
:1057500060FF04C06F5F7F4F8F4F9F4F089557FDCD
:105760009058440F551F59F05F3F71F04795880FCF
:1057700097FB991F61F09F3F79F087950895121666
:1057800013061406551FF2CF4695F1DF08C0161612
:1057900017061806991FF1CF8695710561050894C3
:1057A0000895E894BB2766277727CB0197F90895DA
:1057B000A6E1B0E044E050E00C94ED2B242F0E94D1
:1057C000FC2B252F0E94FC2B0C94E62B0E94FB2B1C
:1057D000272F0C94FC2BDC01CB01FC01F999FECFA7
:1057E00006C0F2BDE1BDF89A319600B40D92415069
:1057F0005040B8F70895262FF999FECF1FBA92BDF1
:1058000081BD20BD0FB6F894FA9AF99A0FBE0196A1
:1058100008952F923F924F925F926F927F928F9254
:105820009F92AF92BF92CF92DF92EF92FF920F932F
:105830001F93CF93DF93CDB7DEB7CA1BDB0B0FB639
:10584000F894DEBF0FBECDBF09942A8839884888F6
:105850005F846E847D848C849B84AA84B984C8848C
:10586000DF80EE80FD800C811B81AA81B981CE0F83
:10587000D11D0FB6F894DEBF0FBECDBFED01089568
:10588000A29FB001B39FC001A39F700D811D112481
:10589000911DB29F700D811D1124911D08955058C6
:1058A000BB27AA270E94672C0C949E2B0E94902B4A
:1058B00038F00E94972B20F039F49F3F19F426F41A
:1058C0000C948D2B0EF4E095E7FB0C94872BE92FBD
:1058D0000E94AF2B58F3BA17620773078407950726
:1058E00020F079F4A6F50C94D12B0EF4E0950B2E54
:1058F000BA2FA02D0B01B90190010C01CA01A00122
:105900001124FF27591B99F0593F50F4503E68F17C
:105910001A16F040A22F232F342F4427585FF3CFBD
:10592000469537952795A795F0405395C9F77EF48E
:105930001F16BA0B620B730B840BBAF09150A1F0D7
:10594000FF0FBB1F661F771F881FC2F70EC0BA0F5D
:10595000621F731F841F48F4879577956795B795E5
:10596000F7959E3F08F0B0CF9395880F08F09927E0
:10597000EE0F9795879508950E94D02C0C949E2B3E
:105980000E94972B58F00E94902B40F029F45F3F23
:1059900029F00C94872B51110C94D22B0C948D2B45
:1059A0000E94AF2B68F39923B1F3552391F3951B14
:1059B000550BBB27AA2762177307840738F09F5F30
:1059C0005F4F220F331F441FAA1FA9F335D00E2E9D
:1059D0003AF0E0E832D091505040E695001CCAF70A
:1059E0002BD0FE2F29D0660F771F881FBB1F2617CD
:1059F00037074807AB07B0E809F0BB0B802DBF01A4
:105A0000FF2793585F4F3AF09E3F510578F00C9472
:105A1000872B0C94D22B5F3FE4F3983ED4F386950A
:105A200077956795B795F7959F5FC9F7880F911D93
:105A30009695879597F90895E1E0660F771F881F7F
:105A4000BB1F621773078407BA0720F0621B730B32
:105A5000840BBA0BEE1F88F7E09508950E94352D50
:105A60006894B1110C94D22B08950E94B72B88F042
:105A70009F5798F0B92F9927B751B0F0E1F0660F12
:105A8000771F881F991F1AF0BA95C9F714C0B13053
:105A900091F00E94D12BB1E008950C94D12B672F87
:105AA000782F8827B85F39F0B93FCCF38695779582
:105AB0006795B395D9F73EF490958095709561956B
:105AC0007F4F8F4F9F4F08950E94F62A08F48FEF63
:105AD0000895A1E21A2EAA1BBB1BFD010DC0AA1F2F
:105AE000BB1FEE1FFF1FA217B307E407F50720F047
:105AF000A21BB30BE40BF50B661F771F881F991FC2
:105B00001A9469F760957095809590959B01AC010A
:105B1000BD01CF010895EE0FFF1F0590F491E02D18
:105B20000994DF93CF931F930F939A9DF02D219F9C
:105B3000F00D8B9DF00D8A9DE02DF10D039FF00D72
:105B4000029FE00DF11D4E9DE00DF11D5E9DF00DDB
:105B50004F9DF00D7F936F93BF92AF925F934F93E2
:105B6000D5010E94402C8B01AC01D7010E94402C32
:105B7000EB01E80FF91FD6010E94E02D2F913F9114
:105B8000D6010E94402CC60FD71FE81FF91FAF9106
:105B9000BF910E94E02D2F913F910E94402CC60F93
:105BA000D71FE81FF91FD6010E94402CE60FF71FF0
:105BB0009801BE01CF010F911F91CF91DF91089500
:105BC0000E94402C460F571FC81FD91F08F431965A
:105BD0000895E894DF93CF93FC01DB010E94402CF1
:105BE0007F936F93E9019A01AC01BF93AF933F9309
:105BF0002F93DF010E94402C26F46C1B7D0B820B3F
:105C0000930B9E01EB01FC010E94E02DAF91BF912F
:105C10002F913F910E94E02DBE01CF01F9012F91FC
:105C20003F91CF91DF910895689401C0E894F92FD6
:105C3000F12B12F00C94482EA0E0B0E0E2E2FEE27C
:105C40000C940F2C092E059422F40E94A42E1123EB
:105C500092F4F0E80F26FFEFE094F0940095109591
:105C6000B094C094D094A194BF0ACF0ADF0AEF0A7F
:105C7000FF0A0F0B1F0B0E94532E07FC0E94A42E3D
:105C8000CDB7DEB7ECE00C942B2C689401C0E894FF
:105C90008F929F92CF93DF930E94532EDF91CF91EB
:105CA0009F908F90089588249924F401E401B0E432
:105CB0009F93AA279A158B049C04ED05FE05CF053A
:105CC000D007A10798F4AD2FDC2FCF2FFE2FE92DA1
:105CD000982C892E982F872F762F652F542F432F9E
:105CE000322F2227B85031F7BF9127C01B2EBF910A
:105CF000BB27220F331F441F551F661F771F881FA6
:105D0000991F881C991CEE1FFF1FCC1FDD1FAA1FA7
:105D1000BB1F8A149B04EC05FD05CE05DF05A0071B
:105D2000B10748F08A189B08EC09FD09CE09DF0984
:105D3000A00BB10B21601A94E1F62EF49401AF018F
:105D4000BE01CD01000C08956095709580959095E9
:105D500030954095509521953F4F4F4F5F4F6F4F76
:105D60007F4F8F4F9F4F0895002E083090F0982F4F
:105D7000872F762F652F542F432F322F222708503D
:105D8000F4CF220F331F441F551F661F771F881F34
:105D9000991F0A95B2F7002D089597FD1094002ED3
:105DA000083098F00850232F342F452F562F672F97
:105DB000782F892F912DF4CF159497958795779506
:105DC000679557954795379527950A95AAF7112412
:105DD000002D08952A0D3B1D4C1D5D1D6E1D7F1D60
:105DE000801F911F08950024A7FD00942A0F301DE5
:105DF000401D501D601D701D801D901D08950024C4
:105E0000A7FD00942A173005400550056005700570
:105E10008005900508950F931F93CF93DF938230F1
:105E2000910510F482E090E0E091C605F091C7057D
:105E300030E020E0B0E0A0E0309799F42115310582
:105E400009F44AC0281B390B24303105D8F58A8162
:105E50009B816115710589F1FB0193838283FE01AA
:105E600011C0408151810281138148175907E0F028
:105E70004817590799F4109761F012960C931297EE
:105E800013961C933296CF01DF91CF911F910F9102
:105E900008950093C6051093C705F4CF2115310569
:105EA00051F04217530738F0A901DB019A01BD01F7
:105EB000DF01F801C1CFEF01F9CF9093C7058093BF
:105EC000C605CDCFFE01E20FF31F819391932250BF
:105ED000310939832883D7CF2091C4053091C50576
:105EE000232B41F420914B0130914C013093C50597
:105EF0002093C4052091490130914A0121153105B3
:105F000041F42DB73EB740914D0150914E01241BF5
:105F1000350BE091C405F091C505E217F307A0F435
:105F20002E1B3F0B2817390778F0AC014E5F5F4FEF
:105F30002417350748F04E0F5F1F5093C505409357
:105F4000C405819391939FCFF0E0E0E09CCFCF9385
:105F5000DF930097E9F0FC01329713821282A0913F
:105F6000C605B091C705ED0130E020E01097A1F41F
:105F700020813181820F931F2091C4053091C50586
:105F80002817390709F061C0F093C505E093C405EF
:105F9000DF91CF910895EA01CE17DF07E8F54A8136
:105FA0005B819E0141155105B1F7E901FB83EA834D
:105FB00049915991C40FD51FEC17FD0761F48081F9
:105FC00091810296840F951FE901998388838281CC
:105FD00093819B838A83F0E0E0E012968D919C91FF
:105FE00013970097B9F52D913C911197CD01029629
:105FF000820F931F2091C4053091C50528173907DA
:1060000039F6309751F51092C7051092C605B09336
:10601000C505A093C405BCCFD383C2834081518101
:10602000840F951FC817D90761F44E5F5F4F8881B1
:106030009981480F591F518340838A819B819383A3
:1060400082832115310509F0B0CFF093C705E093A5
:10605000C6059ECFFD01DC01C0CF13821282D7CFCF
:10606000B0E0A0E0E6E3F0E30C940B2C8C01009789
:1060700051F4CB010E940B2F8C01C801CDB7DEB7C4
:10608000E0E10C94272CFC01E60FF71F9C01225045
:106090003109E217F30708F49DC0D901CD91DC91D5
:1060A0001197C617D70798F0C530D10530F3CE0148
:1060B00004978617970708F3C61BD70B2297C1933F
:1060C000D1936D937C93CF010E94A72FD6CF5B0114
:1060D000AC1ABD0A4C018C0E9D1EA091C605B09154
:1060E000C705512C412CF12CE12C109731F58091F2
:1060F000C4059091C5058815990509F05CC0461640
:10610000570608F058C08091490190914A010097C4
:1061100041F48DB79EB740914D0150914E01841BC3
:10612000950BE817F90708F055C0F093C505E09303
:10613000C405F90171836083A0CF8D919C91119763
:1061400012966C90129713967C901397A815B90528
:1061500059F56C0142E0C40ED11CCA14DB0420F1D5
:10616000AC014A195B09DA011296159780F0628238
:10617000738251834083D9016D937C93E114F104C0
:1061800071F0D7011396FC93EE93129776CF229677
:106190008C0F9D1FF90191838083F301EFCFF09362
:1061A000C705E093C60569CF4816590608F42C01C7
:1061B0007D01D3019ACFCB010E940B2F7C01009768
:1061C00049F0AE01B8010E94ED30C8010E94A72F2E
:1061D000870153CF10E000E050CFFB01DC0102C08B
:1061E00001900D9241505040D8F70895FB01DC0119
:1061F0008D91019080190110D9F3990B0895FB013D
:10620000DC0101900D920020E1F7089510E0C2E654
:10621000D0E004C0FE010E948B2D2196C336D10729
:10622000C9F7F894FFCF0300E8030000030080964D
:10623000980040787D011F151F1B1F1F110E1F1591
:106240001F1B1F1F111F1F151F1B1F0E111F1F15A7
:106250001F1B0E0E111F0100C0CF6A0001008096A7
:1062600098008096980080969800010000803F007A
:1062700000C80580000002040003000110030200B2
:1062800000030201000600040006050020060504C4
:106290000000000000A107F8062E07EE075F073D8B
:1062A00007510700000000C70A9A0A4A0B770A8DB7
:1062B00000870A780A1400FA002C01000000001080
:1062C0000FF8064A0BF7062053007874616C202003
:1062D000005553422020004C534220200043414CA3
:1062E0004942524152006F4B3D4231207361693D3A
:1062F0004232200043414C494252415220585441BD
:106300004C204652004D65646972206672657120AA
:10631000434C4B300051646F206F6B20636C69718C
:10632000756520423100416A75737465206671207D
:106330006D65646964610020657370657265202015
:106340002020202020200042323D5341492042316C
:106350003D4752415641200020204752415641447A
:106360004F202020202020200042323D5341492050
:106370002020202020202020202000414A55535456
:1063800045204C53420056464F20656D2031373131
:1063900030306B487A002042464F20656D20004126
:1063A0004A2E20727569646F20616C746F00414AD7
:1063B00020544F4D202B20475241564500456E63D7
:1063C0006F6E74726520756D2051534F2000436FBE
:1063D0006D2030206F7520356B487A2020200041D9
:1063E0004A555354452041474F52412042464F00A1
:1063F00041544520464943415220434C41524F208D
:106400000020657370657265004232205341492057
:10641000423120475241564120200020204752411E
:106420005641444F202020202000414A55535445D6
:10643000205553420056464F20656D20323930308A
:106440006B487A00456E636F6E74726520756D20BF
:1064500051534F00436F6D2030206F7520356B48CE
:106460007A200051646F206F6B20636C69717565D1
:106470002042320042323D5341492042313D475291
:1064800041564120200036202000372020003820AF
:106490002000392020002B3130002B3230004357B0
:1064A000200046543800475241564120415455413E
:1064B0004C2046524551004F4B3D4231207361699B
:0664C0003D423220000005
:107E0000112484B714BE81FFF0D085E080938100F7
:107E100082E08093C00088E18093C10086E0809377
:107E2000C20080E18093C4008EE0C9D0259A86E02C
:107E300020E33CEF91E0309385002093840096BBD3
:107E4000B09BFECF1D9AA8958150A9F7CC24DD24C4
:107E500088248394B5E0AB2EA1E19A2EF3E0BF2EE7
:107E6000A2D0813461F49FD0082FAFD0023811F036
:107E7000013811F484E001C083E08DD089C08234E0
:107E800011F484E103C0853419F485E0A6D080C0E4
:107E9000853579F488D0E82EFF2485D0082F10E0AE
:107EA000102F00270E291F29000F111F8ED06801E7
:107EB0006FC0863521F484E090D080E0DECF843638
:107EC00009F040C070D06FD0082F6DD080E0C81688
:107ED00080E7D80618F4F601B7BEE895C0E0D1E017
:107EE00062D089930C17E1F7F0E0CF16F0E7DF06D8
:107EF00018F0F601B7BEE89568D007B600FCFDCFD4
:107F0000A601A0E0B1E02C9130E011968C91119780
:107F100090E0982F8827822B932B1296FA010C0160
:107F200087BEE89511244E5F5F4FF1E0A038BF0790
:107F300051F7F601A7BEE89507B600FCFDCF97BE46
:107F4000E89526C08437B1F42ED02DD0F82E2BD052
:107F50003CD0F601EF2C8F010F5F1F4F84911BD097
:107F6000EA94F801C1F70894C11CD11CFA94CF0C13
:107F7000D11C0EC0853739F428D08EE10CD085E9AC
:107F80000AD08FE07ACF813511F488E018D01DD067
:107F900080E101D065CF982F8091C00085FFFCCF94
:107FA0009093C60008958091C00087FFFCCF809118
:107FB000C00084FD01C0A8958091C6000895E0E648
:107FC000F0E098E1908380830895EDDF803219F02E
:107FD00088E0F5DFFFCF84E1DECF1F93182FE3DFCA
:107FE0001150E9F7F2DF1F91089580E0E8DFEE27F6
:047FF000FF270994CA
:027FFE00040479
:00000001FF
